Stack Allocation = 16384 bytes

 SPSVR16

 Start     Length     Name                   Class
 0001:0000 03C12H     SEG_CODE_TEXT          CODE
 0001:3C12 00000H     HATCH_TEXT             CODE
 0001:3C12 00000H     OLE2UI_TEXT            CODE
 0001:3C12 00000H     OLEUTL_TEXT            CODE
 0001:3C12 00000H     ICONBOX_TEXT           CODE
 0001:3C12 00000H     OBJFDBK_TEXT           CODE
 0001:3C12 00000H     OLESTD_TEXT            CODE
 0001:3C12 00000H     RESIMAGE_TEXT          CODE
 0001:3C12 00000H     DRAWICON_TEXT          CODE
 0001:3C12 00000H     TARGTDEV_TEXT          CODE
 0001:3C12 00000H     REGDB_TEXT             CODE
 0001:3C12 021FFH     _TEXT                  CODE
 0001:5E20 02F35H     COMDAT_SEG1            CODE
 0002:0000 00010H     NULL                   BEGDATA
 0002:0010 010B2H     _DATA                  DATA
 0002:10C2 0000EH     CDATA                  DATA
 0002:10D0 00000H     XIB                    DATA
 0002:10D0 00004H     XI                     DATA
 0002:10D4 00000H     XIE                    DATA
 0002:10D4 00000H     XIFB                   DATA
 0002:10D4 00000H     XIF                    DATA
 0002:10D4 00000H     XIFE                   DATA
 0002:10D4 00000H     XPB                    DATA
 0002:10D4 00000H     XP                     DATA
 0002:10D4 00000H     XPE                    DATA
 0002:10D4 00000H     XCB                    DATA
 0002:10D4 00000H     XC                     DATA
 0002:10D4 00000H     XCE                    DATA
 0002:10D4 00000H     XCFB                   DATA
 0002:10D4 00000H     XCFCRT                 DATA
 0002:10D4 00000H     XCF                    DATA
 0002:10D4 00000H     XCFE                   DATA
 0002:10D4 00000H     XIFCB                  DATA
 0002:10D4 00000H     XIFU                   DATA
 0002:10D4 00000H     XIFL                   DATA
 0002:10D4 00000H     XIFM                   DATA
 0002:10D4 00000H     XIFCE                  DATA
 0002:10D4 00000H     DBDATA                 DATA
 0002:10D4 00014H     CONST                  CONST
 0002:10E8 00008H     HDR                    MSG
 0002:10F0 003EEH     MSG                    MSG
 0002:14DE 00002H     PAD                    MSG
 0002:14E0 00001H     EPAD                   MSG
 0002:14E2 00A48H     _BSS                   BSS
 0002:1F2A 00000H     XOB                    BSS
 0002:1F2A 00000H     XO                     BSS
 0002:1F2A 00000H     XOE                    BSS
 0002:1F2A 00000H     XOFB                   BSS
 0002:1F2A 00000H     XOF                    BSS
 0002:1F2A 00000H     XOFE                   BSS
 0002:1F30 00018H     c_common               BSS

 Origin   Group
 0002:0   DGROUP

 Address   Export                  Alias

 0001:510C ___ExportedStub         ___ExportedStub

  Address         Publics by Name

 0001:5212       $i8_output
 0001:5538       $i8_tpwr10
 0001:0000       ??0CSimpSvrApp@@REC@XZ
 0001:07DC       ??0CSimpSvrDoc@@REC@PEVCSimpSvrApp@@I@Z
 0001:2A46       ??0CSimpSvrObj@@REC@PEVCSimpSvrDoc@@@Z
 0001:5EAE       ??0IOleWindow@@REC@XZ
 0001:5ED6       ??0IPersist@@REC@XZ
 0001:006E       ??1CSimpSvrApp@@REC@XZ
 0001:0832       ??1CSimpSvrDoc@@REC@XZ
 0001:2CBA       ??1CSimpSvrObj@@REC@XZ
 0001:3CFC       ??2@ZAPEXI@Z
 0001:3CEA       ??3@ZAXPEX@Z
 0001:5E62       ??_7CClassFactory@@6F@
 0001:5F3A       ??_7CDataObject@@6F@
 0001:6116       ??_7CExternalConnection@@6F@
 0001:6136       ??_7COleInPlaceActiveObject@@6F@
 0001:60BE       ??_7COleInPlaceObject@@6F@
 0001:5FC2       ??_7COleObject@@6F@
 0001:6022       ??_7CPersistStorage@@6F@
 0001:5E76       ??_7CSimpSvrApp@@6F@
 0001:5E82       ??_7CSimpSvrDoc@@6F@
 0001:612A       ??_7CSimpSvrObj@@6F@
 0001:5E42       ??_7IClassFactory@@6F@
 0001:5F6A       ??_7IDataObject@@6F@
 0001:5EFE       ??_7IExternalConnection@@6F@
 0001:5F9A       ??_7IOleInPlaceActiveObject@@6F@
 0001:60F2       ??_7IOleInPlaceObject@@6F@
 0001:605E       ??_7IOleObject@@6F@
 0001:604A       ??_7IOleWindow@@6F@
 0001:60E2       ??_7IPersist@@6F@
 0001:5F12       ??_7IPersistStorage@@6F@
 0001:5E56       ??_7IUnknown@@6F@
 0001:6BD4       ??_C@_00A@?$AA@
 0001:6BD6       ??_C@_03NAME@?4?4?4?$AA@
 0001:6BE4       ??_C@_04FOAE@?$CFd?$CF?$CF?$AA@
 0001:7DCC       ??_C@_04MOFI@?$CFs?$CFd?$AA@
 0001:7D88       ??_C@_05FGFK@CLSID?$AA@
 0001:8D10       ??_C@_06HFAC@CLSID?2?$AA@
 0001:7E04       ??_C@_06KAHL@?$EA?$CFs?$CB?$CFs?$AA@
 0001:64DE       ??_C@_07CIAP@windows?$AA@
 0001:7D98       ??_C@_07CPIP@Package?$AA@
 0001:897A       ??_C@_07LGIJ@DISPLAY?$AA@
 0001:8D06       ??_C@_08BJKM@CLSID?2?$CFs?$AA@
 0001:6B8C       ??_C@_08NJLM@FileName?$AA@
 0001:6BDA       ??_C@_09DKHB@Structure?$AA@
 0001:7D8E       ??_C@_09JJAI@Linked?5?$CFs?$AA@
 0001:6EE8       ??_C@_09LHIP@Embedding?$AA@
 0001:6B82       ??_C@_09NJ@OwnerLink?$AA@
 0001:6B66       ??_C@_0BA@IEJA@Embedded?5Object?$AA@
 0001:8D18       ??_C@_0BA@LJEI@?2AuxUserType?2?$CFd?$AA@
 0001:6AD8       ??_C@_0BB@PGGH@OLEUI_MSG_BROWSE?$AA@
 0001:6B2E       ??_C@_0BC@GMEI@Object?5Descriptor?$AA@
 0001:6B00       ??_C@_0BD@HNAP@commdlg_FileNameOK?$AA@
 0001:6AC4       ??_C@_0BE@FEHN@OLEUI_MSG_ENDDIALOG?$AA@
 0001:6AEA       ??_C@_0BF@COIE@OLEUI_MSG_CHANGEICON?$AA@
 0001:64C8       ??_C@_0BG@FPGD@oleinplaceborderwidth?$AA@
 0001:6B40       ??_C@_0BH@FOOO@Link?5Source?5Descriptor?$AA@
 0001:6B14       ??_C@_0BK@LOCD@OLEUI_MSG_CLOSEBUSYDIALOG?$AA@
 0001:5E8E       ??_C@_0CA@JEOC@In?5CClassFactory?8s?5Destructor?$AN?6?$AA@
 0001:8D34       ??_C@_0CB@FCAE@CLSID?2?$CFs?2DataFormats?2DefaultFile@
 0001:5E20       ??_C@_0CB@GPOM@In?5CClassFactory?8s?5Constructor?$AN?6@
 0001:6BAE       ??_C@_0CG@HCKA@resource?5read?50x?$CFX?0?5my?5value?5is?5@
 0001:7DA0       ??_C@_0CL@HONB@ERROR?3?5INTERFACE?5METHOD?5NOT?5IMPL@
 0001:7DD2       ??_C@_0DC@GEMK@OleStdCreateTempFileMoniker?3?5Mon@
 0001:7D4E       ??_C@_0DJ@NHNH@OleStdSwitchDisplayAspect?3?5Cache@
 0001:8D28       ??_C@_0M@BODG@?2MiscStatus?$AA@
 0001:6BA2       ??_C@_0M@GHPL@ole2uiIBCls?$AA@
 0001:6B76       ??_C@_0M@KPGD@Link?5Source?$AA@
 0001:6B96       ??_C@_0M@MBIN@ole2uiRICls?$AA@
 0001:64BA       ??_C@_0N@JEKA@Hatch?5Window?$AA@
 0001:6B58       ??_C@_0N@LHIH@Embed?5Source?$AA@
 0001:6AA6       ??_C@_0N@OCMF@VERIFICATION?$AA@
 0001:6AB4       ??_C@_0P@LMIA@OLEUI_MSG_HELP?$AA@
 0001:3B3E       ?About@@ZCHIIGJ@Z
 0001:1434       ?AddConnection@CExternalConnection@@VEAKKK@Z
 0001:358C       ?AddFrameLevelUI@CSimpSvrObj@@RECXXZ
 0001:0EEE       ?AddRef@CClassFactory@@VEAKXZ
 0001:1046       ?AddRef@CDataObject@@VEAKXZ
 0001:13CC       ?AddRef@CExternalConnection@@VEAKXZ
 0001:1516       ?AddRef@COleInPlaceActiveObject@@VEAKXZ
 0001:1714       ?AddRef@COleInPlaceObject@@VEAKXZ
 0001:1A64       ?AddRef@COleObject@@VEAKXZ
 0001:2278       ?AddRef@CPersistStorage@@VEAKXZ
 0001:0138       ?AddRef@CSimpSvrApp@@VEAKXZ
 0001:08E0       ?AddRef@CSimpSvrDoc@@VEAKXZ
 0001:29A6       ?AddRef@CSimpSvrObj@@VEAKXZ
 0001:1B5A       ?Advise@COleObject@@VEAPEXPEUIAdviseSink@@PEK@Z
 0001:34D2       ?AssembleMenus@CSimpSvrObj@@RECXXZ
 0001:1DC6       ?Close@COleObject@@VEAPEXK@Z
 0001:0A78       ?Close@CSimpSvrDoc@@RECXXZ
 0001:15F8       ?ContextSensitiveHelp@COleInPlaceActiveObject@@VEAPEXH@Z
 0001:19EC       ?ContextSensitiveHelp@COleInPlaceObject@@VEAPEXH@Z
 0001:0710       ?Create@CSimpSvrDoc@@TAPEV1@PEVCSimpSvrApp@@PEUtagRECT@@I@Z
 0001:0F76       ?CreateInstance@CClassFactory@@VEAPEXPEUIUnknown@@AFUGUID@@PEPEX@Z
 0001:09F0       ?CreateObject@CSimpSvrDoc@@RECPEXAFUGUID@@PEPEX@Z
 0001:259C       ?CreateStreams@CPersistStorage@@RECXPEUIStorage@@@Z
 0001:27C0       ?CreateStreams@CPersistStorage@@RECXPEUIStorage@@PEPEUIStream@@1@Z
 0001:1108       ?DAdvise@CDataObject@@VEAPEXPEUtagFORMATETC@@KPEUIAdviseSink@@PEK@Z
 0001:37DE       ?DeactivateUI@CSimpSvrObj@@RECXXZ
 0001:36F0       ?DisassembleMenus@CSimpSvrObj@@RECXXZ
 0001:3B76       ?DocWndProc@@ZCJIIIJ@Z
 0001:321C       ?DoInPlaceActivate@CSimpSvrObj@@RECHJ@Z
 0001:3642       ?DoInPlaceHide@CSimpSvrObj@@RECXXZ
 0001:1BD0       ?DoVerb@COleObject@@VEAPEXJPEUtagMSG@@PEUIOleClientSite@@JIPFUtagRECT@@@Z
 0001:2D7E       ?Draw@CSimpSvrObj@@RECXIH@Z
 0001:11F4       ?DUnadvise@CDataObject@@VEAPEXK@Z
 0001:16B6       ?EnableModeless@COleInPlaceActiveObject@@VEAPEXH@Z
 0001:20DA       ?EnumAdvise@COleObject@@VEAPEXPEPEUIEnumSTATDATA@@@Z
 0001:134E       ?EnumDAdvise@CDataObject@@VEAPEXPEPEUIEnumSTATDATA@@@Z
 0001:1328       ?EnumFormatEtc@CDataObject@@VEAPEXKPEPEUIEnumFORMATETC@@@Z
 0001:1E2E       ?EnumVerbs@COleObject@@VEAPEXPEPEUIEnumOLEVERB@@@Z
 0002:0DD2       ?fBeVerbose@@3HE
 0001:01A8       ?fInitApplication@CSimpSvrApp@@RECHI@Z
 0001:0274       ?fInitInstance@CSimpSvrApp@@RECHIHPEUCClassFactory@@@Z
 0001:1270       ?GetCanonicalFormatEtc@CDataObject@@VEAPEXPEUtagFORMATETC@@0@Z
 0001:235A       ?GetClassID@CPersistStorage@@VEAPEXPEUGUID@@@Z
 0001:1E4A       ?GetClientSite@COleObject@@VEAPEXPEPEUIOleClientSite@@@Z
 0001:201E       ?GetClipboardData@COleObject@@VEAPEXKPEPEUIDataObject@@@Z
 0001:1172       ?GetData@CDataObject@@VEAPEXPEUtagFORMATETC@@PEUtagSTGMEDIUM@@@Z
 0001:1252       ?GetDataHere@CDataObject@@VEAPEXPEUtagFORMATETC@@PEUtagSTGMEDIUM@@@Z
 0001:1D22       ?GetExtent@COleObject@@VEAPEXKPEUtagSIZEL@@@Z
 0001:2EFE       ?GetMetaFilePict@CSimpSvrObj@@RECIXZ
 0001:211C       ?GetMiscStatus@COleObject@@VEAPEXKPEK@Z
 0001:1FB0       ?GetMoniker@COleObject@@VEAPEXKKPEPEUIMoniker@@@Z
 0001:2062       ?GetUserClassID@COleObject@@VEAPEXPEUGUID@@@Z
 0001:20A0       ?GetUserType@COleObject@@VEAPEXKPEPED@Z
 0001:15C8       ?GetWindow@COleInPlaceActiveObject@@VEAPEXPEI@Z
 0001:19BC       ?GetWindow@COleInPlaceObject@@VEAPEXPEI@Z
 0001:2578       ?HandsOffStorage@CPersistStorage@@VEAPEXXZ
 0001:06EC       ?HideAppWnd@CSimpSvrApp@@RECXXZ
 0001:0E1C       ?HideDocWnd@CSimpSvrDoc@@RECXXZ
 0001:0E32       ?HideHatchWnd@CSimpSvrDoc@@RECXXZ
 0001:2002       ?InitFromData@COleObject@@VEAPEXPEUIDataObject@@HK@Z
 0001:22E0       ?InitNew@CPersistStorage@@VEAPEXPEUIStorage@@@Z
 0001:177C       ?InPlaceDeactivate@COleInPlaceObject@@VEAPEXXZ
 0001:255E       ?IsDirty@CPersistStorage@@VEAPEXXZ
 0001:067C       ?IsInPlaceActive@CSimpSvrApp@@RECHXZ
 0001:2048       ?IsUpToDate@COleObject@@VEAPEXXZ
 0001:0432       ?lCommandHandler@CSimpSvrApp@@RECJIIIJ@Z
 0001:05E2       ?lCreateDoc@CSimpSvrApp@@RECJIIIJ@Z
 0001:24B0       ?Load@CPersistStorage@@VEAPEXPEUIStorage@@@Z
 0001:315C       ?LoadFromStorage@CSimpSvrObj@@RECXXZ
 0001:0FDA       ?LockServer@CClassFactory@@VEAPEXH@Z
 0002:14E6       ?lpClassFactory@@3PEUCClassFactory@@E
 0002:14E2       ?lpCSimpSvrApp@@3PEVCSimpSvrApp@@E
 0001:0980       ?lResizeDoc@CSimpSvrDoc@@RECJPEUtagRECT@@@Z
 0001:05B4       ?lSizeHandler@CSimpSvrApp@@RECJIIIJ@Z
 0001:39FC       ?MainWndProc@@ZCJIIIJ@Z
 0001:157E       ?OnDocWindowActivate@COleInPlaceActiveObject@@VEAPEXH@Z
 0001:15AE       ?OnFrameWindowActivate@COleInPlaceActiveObject@@VEAPEXH@Z
 0001:215C       ?OpenEdit@COleObject@@RECXPEUIOleClientSite@@@Z
 0001:265A       ?OpenStreams@CPersistStorage@@RECXPEUIStorage@@@Z
 0001:0618       ?PaintApp@CSimpSvrApp@@RECXI@Z
 0001:09AA       ?PaintDoc@CSimpSvrDoc@@RECXI@Z
 0001:063C       ?ParseCmdLine@CSimpSvrApp@@RECXPED@Z
 0001:10AE       ?QueryGetData@CDataObject@@VEAPEXPEUtagFORMATETC@@@Z
 0001:0E48       ?QueryInterface@CClassFactory@@VEAPEXAFUGUID@@PEPEX@Z
 0001:100A       ?QueryInterface@CDataObject@@VEAPEXAFUGUID@@PEPEX@Z
 0001:1390       ?QueryInterface@CExternalConnection@@VEAPEXAFUGUID@@PEPEX@Z
 0001:14DA       ?QueryInterface@COleInPlaceActiveObject@@VEAPEXAFUGUID@@PEPEX@Z
 0001:16D0       ?QueryInterface@COleInPlaceObject@@VEAPEXAFUGUID@@PEPEX@Z
 0001:1A28       ?QueryInterface@COleObject@@VEAPEXAFUGUID@@PEPEX@Z
 0001:223C       ?QueryInterface@CPersistStorage@@VEAPEXAFUGUID@@PEPEX@Z
 0001:00AC       ?QueryInterface@CSimpSvrApp@@VEAPEXAFUGUID@@PEPEX@Z
 0001:0872       ?QueryInterface@CSimpSvrDoc@@VEAPEXAFUGUID@@PEPEX@Z
 0001:281C       ?QueryInterface@CSimpSvrObj@@VEAPEXAFUGUID@@PEPEX@Z
 0001:1A0A       ?ReactivateAndUndo@COleInPlaceObject@@VEAPEXXZ
 0001:0F12       ?Release@CClassFactory@@VEAKXZ
 0001:107A       ?Release@CDataObject@@VEAKXZ
 0001:1400       ?Release@CExternalConnection@@VEAKXZ
 0001:154A       ?Release@COleInPlaceActiveObject@@VEAKXZ
 0001:1748       ?Release@COleInPlaceObject@@VEAKXZ
 0001:1A98       ?Release@COleObject@@VEAKXZ
 0001:22AC       ?Release@CPersistStorage@@VEAKXZ
 0001:015C       ?Release@CSimpSvrApp@@VEAKXZ
 0001:091C       ?Release@CSimpSvrDoc@@VEAKXZ
 0001:29E2       ?Release@CSimpSvrObj@@VEAKXZ
 0001:146C       ?ReleaseConnection@CExternalConnection@@VEAKKKH@Z
 0001:2716       ?ReleaseStreamsAndStorage@CPersistStorage@@RECXXZ
 0001:1632       ?ResizeBorder@COleInPlaceActiveObject@@VEAPEXPFUtagRECT@@PEUIOleInPlaceUIWindow@@H@Z
 0001:238A       ?Save@CPersistStorage@@VEAPEXPEUIStorage@@H@Z
 0001:23DA       ?SaveCompleted@CPersistStorage@@VEAPEXPEUIStorage@@@Z
 0001:2FB8       ?SaveToStorage@CSimpSvrObj@@RECXPEUIStorage@@H@Z
 0001:374E       ?SendOnDataChange@CSimpSvrObj@@RECXXZ
 0001:1ACC       ?SetClientSite@COleObject@@VEAPEXPEUIOleClientSite@@@Z
 0001:2142       ?SetColorScheme@COleObject@@VEAPEXPEUtagLOGPALETTE@@@Z
 0001:130A       ?SetData@CDataObject@@VEAPEXPEUtagFORMATETC@@PEUtagSTGMEDIUM@@H@Z
 0001:20BC       ?SetExtent@COleObject@@VEAPEXKPEUtagSIZEL@@@Z
 0001:1BB6       ?SetHostNames@COleObject@@VEAPEXPFD0@Z
 0001:1E7E       ?SetMoniker@COleObject@@VEAPEXKPEUIMoniker@@@Z
 0001:1854       ?SetObjectRects@COleInPlaceObject@@VEAPEXPFUtagRECT@@0@Z
 0001:0664       ?SetStatusText@CSimpSvrApp@@RECXXZ
 0001:0DA0       ?SetStatusText@CSimpSvrDoc@@RECXXZ
 0001:06BA       ?ShowAppWnd@CSimpSvrApp@@RECXH@Z
 0001:0DE4       ?ShowDocWnd@CSimpSvrDoc@@RECXXZ
 0001:0E06       ?ShowHatchWnd@CSimpSvrDoc@@RECXXZ
 0001:1616       ?TranslateAccelerator@COleInPlaceActiveObject@@VEAPEXPEUtagMSG@@@Z
 0001:182A       ?UIDeactivate@COleInPlaceObject@@VEAPEXXZ
 0001:1DF4       ?Unadvise@COleObject@@VEAPEXK@Z
 0001:1D9C       ?Update@COleObject@@VEAPEXXZ
 0000:0000  Imp  ANSINEXT             (USER.472)
 0000:0000  Imp  ANSITOOEM            (KEYBOARD.5)
 0000:0000  Imp  BEGINPAINT           (USER.39)
 0000:0000  Imp  BITBLT               (GDI.34)
 0000:0000  Imp  CLOSEMETAFILE        (GDI.126)
 0000:0000  Imp  CLSIDFROMPROGID      (COMPOBJ.61)
 0000:0000  Imp  CODISCONNECTOBJECT   (COMPOBJ.15)
 0000:0000  Imp  CODOSDATETIMETOFILETIME (COMPOBJ.31)
 0000:0000  Imp  COFILETIMENOW        (COMPOBJ.82)
 0000:0000  Imp  COGETMALLOC          (COMPOBJ.4)
 0000:0000  Imp  COISOLE1CLASS        (COMPOBJ.36)
 0000:0000  Imp  COLOCKOBJECTEXTERNAL (COMPOBJ.63)
 0000:0000  Imp  COPYRECT             (USER.74)
 0000:0000  Imp  COREGISTERCLASSOBJECT (COMPOBJ.5)
 0000:0000  Imp  COREVOKECLASSOBJECT  (COMPOBJ.6)
 0000:0000  Imp  COTREATASCLASS       (COMPOBJ.66)
 0000:0000  Imp  CREATEBINDCTX        (OLE2.26)
 0000:0000  Imp  CREATEBITMAP         (GDI.48)
 0000:0000  Imp  CREATEBRUSHINDIRECT  (GDI.50)
 0000:0000  Imp  CREATECOMPATIBLEBITMAP (GDI.51)
 0000:0000  Imp  CREATECOMPATIBLEDC   (GDI.52)
 0000:0000  Imp  CREATEDATAADVISEHOLDER (OLE2.39)
 0000:0000  Imp  CREATEDC             (GDI.53)
 0000:0000  Imp  CREATEFILEMONIKER    (OLE2.28)
 0001:61C4       CREATEHATCHWINDOW
 0000:0000  Imp  CREATEIC             (GDI.153)
 0000:0000  Imp  CREATEICON           (USER.407)
 0000:0000  Imp  CREATEILOCKBYTESONHGLOBAL (OLE2.54)
 0000:0000  Imp  CREATEMENU           (USER.151)
 0000:0000  Imp  CREATEMETAFILE       (GDI.125)
 0000:0000  Imp  CREATEOLEADVISEHOLDER (OLE2.38)
 0000:0000  Imp  CREATEPATTERNBRUSH   (GDI.60)
 0000:0000  Imp  CREATEPEN            (GDI.61)
 0000:0000  Imp  CREATEPOPUPMENU      (USER.415)
 0000:0000  Imp  CREATESOLIDBRUSH     (GDI.66)
 0000:0000  Imp  CREATESTREAMONHGLOBAL (OLE2.84)
 0000:0000  Imp  CREATEWINDOW         (USER.41)
 0000:0000  Imp  DEFWINDOWPROC        (USER.107)
 0000:0000  Imp  DELETEDC             (GDI.68)
 0000:0000  Imp  DELETEMENU           (USER.413)
 0000:0000  Imp  DELETEMETAFILE       (GDI.127)
 0000:0000  Imp  DELETEOBJECT         (GDI.69)
 0000:0000  Imp  DESTROYMENU          (USER.152)
 0000:0000  Imp  DESTROYWINDOW        (USER.53)
 0000:0000  Imp  DIALOGBOX            (USER.87)
 0000:0000  Imp  DIALOGBOXPARAM       (USER.239)
 0000:0000  Imp  DISPATCHMESSAGE      (USER.114)
 0000:0000  Imp  DOS3CALL             (KERNEL.102)
 0000:0000  Imp  ENDDIALOG            (USER.88)
 0000:0000  Imp  ENDPAINT             (USER.40)
 0000:0000  Imp  ENUMMETAFILE         (GDI.175)
 0001:84BE       ENUMMETAFILEEXTRACTICON
 0001:86EA       ENUMMETAFILEEXTRACTICONSOURCE
 0001:83E0       ENUMMETAFILEEXTRACTLABEL
 0001:8364       ENUMMETAFILEICONDRAW
 0000:0000  Imp  FATALAPPEXIT         (KERNEL.137)
 0000:0000  Imp  FATALEXIT            (KERNEL.1)
 0000:FE32  Abs  FIARQQ
 0000:0E32  Abs  FICRQQ
 0000:5C32  Abs  FIDRQQ
 0000:1632  Abs  FIERQQ
 0000:0000  Imp  FILLRECT             (USER.81)
 0000:0000  Imp  FINDRESOURCE         (KERNEL.60)
 0000:0632  Abs  FISRQQ
 0000:A23D  Abs  FIWRQQ
 0000:4000  Abs  FJARQQ
 0000:C000  Abs  FJCRQQ
 0000:8000  Abs  FJSRQQ
 0000:0000  Imp  FRAMERECT            (USER.83)
 0000:0000  Imp  FREEPROCINSTANCE     (KERNEL.52)
 0000:0000  Imp  FREERESOURCE         (KERNEL.63)
 0000:0000  Imp  GETBITMAPBITS        (GDI.74)
 0000:0000  Imp  GETBKCOLOR           (GDI.75)
 0000:0000  Imp  GETCLASSFILE         (OLE2.57)
 0000:0000  Imp  GETCLIENTRECT        (USER.33)
 0000:0000  Imp  GETDC                (USER.66)
 0000:0000  Imp  GETDEVICECAPS        (GDI.80)
 0000:0000  Imp  GETDLGITEM           (USER.91)
 0000:0000  Imp  GETDLGITEMTEXT       (USER.93)
 0000:0000  Imp  GETDOSENVIRONMENT    (KERNEL.131)
 0001:6232       GETHATCHRECT
 0001:620E       GETHATCHWIDTH
 0000:0000  Imp  GETMENU              (USER.157)
 0000:0000  Imp  GETMESSAGE           (USER.108)
 0000:0000  Imp  GETMODULEFILENAME    (KERNEL.49)
 0000:0000  Imp  GETOBJECT            (GDI.82)
 0000:0000  Imp  GETPARENT            (USER.46)
 0000:0000  Imp  GETPROFILEINT        (KERNEL.57)
 0000:0000  Imp  GETPROP              (USER.25)
 0000:0000  Imp  GETRUNNINGOBJECTTABLE (OLE2.30)
 0000:0000  Imp  GETSTOCKOBJECT       (GDI.87)
 0000:0000  Imp  GETSUBMENU           (USER.159)
 0000:0000  Imp  GETSYSCOLOR          (USER.180)
 0000:0000  Imp  GETSYSTEMMETRICS     (USER.179)
 0000:0000  Imp  GETVERSION           (KERNEL.3)
 0000:0000  Imp  GETWINDOWWORD        (USER.133)
 0000:0000  Imp  GLOBALALLOC          (KERNEL.15)
 0000:0000  Imp  GLOBALFREE           (KERNEL.17)
 0000:0000  Imp  GLOBALLOCK           (KERNEL.18)
 0000:0000  Imp  GLOBALREALLOC        (KERNEL.16)
 0000:0000  Imp  GLOBALSIZE           (KERNEL.20)
 0000:0000  Imp  GLOBALUNLOCK         (KERNEL.19)
 0001:63D6       HATCHWNDPROC
 0001:6F6A       ICONBOXWNDPROC
 0000:0000  Imp  INFLATERECT          (USER.78)
 0000:0000  Imp  INITAPP              (USER.5)
 0000:0000  Imp  INITTASK             (KERNEL.91)
 0000:0000  Imp  INSERTMENU           (USER.410)
 0000:0000  Imp  INTERSECTRECT        (USER.79)
 0000:0000  Imp  INVALIDATERECT       (USER.125)
 0000:0000  Imp  INVERTRECT           (USER.82)
 0000:0000  Imp  ISBADREADPTR         (KERNEL.334)
 0000:0000  Imp  ISDBCSLEADBYTE       (KERNEL.207)
 0000:0000  Imp  ISDIALOGMESSAGE      (USER.90)
 0000:0000  Imp  ISEQUALGUID          (COMPOBJ.18)
 0000:0000  Imp  ISWINDOW             (USER.47)
 0000:0000  Imp  KILLTIMER            (USER.12)
 0000:0000  Imp  LOADBITMAP           (USER.175)
 0000:0000  Imp  LOADCURSOR           (USER.173)
 0000:0000  Imp  LOADICON             (USER.174)
 0000:0000  Imp  LOADRESOURCE         (KERNEL.61)
 0000:0000  Imp  LOADSTRING           (USER.176)
 0000:0000  Imp  LOCKRESOURCE         (KERNEL.62)
 0000:0000  Imp  LOCKSEGMENT          (KERNEL.23)
 0000:0000  Imp  LSTRCAT              (KERNEL.89)
 0000:0000  Imp  LSTRCMP              (USER.430)
 0000:0000  Imp  LSTRCMPI             (USER.471)
 0000:0000  Imp  LSTRCPY              (KERNEL.88)
 0000:0000  Imp  LSTRCPYN             (KERNEL.353)
 0000:0000  Imp  LSTRLEN              (KERNEL.90)
 0000:0000  Imp  MAKEPROCINSTANCE     (KERNEL.51)
 0000:0000  Imp  MESSAGEBOX           (USER.1)
 0000:0000  Imp  MKPARSEDISPLAYNAME   (OLE2.23)
 0000:0000  Imp  MOVEWINDOW           (USER.56)
 0000:0000  Imp  MULDIV               (GDI.128)
 0000:0000  Imp  OFFSETRECT           (USER.77)
 0000:0000  Imp  OLEBUILDVERSION      (OLE2.1)
 0000:0000  Imp  OLECREATEMENUDESCRIPTOR (OLE2.40)
 0000:0000  Imp  OLEDESTROYMENUDESCRIPTOR (OLE2.42)
 0000:0000  Imp  OLEDUPLICATEDATA     (OLE2.51)
 0000:0000  Imp  OLEINITIALIZE        (OLE2.2)
 0000:0000  Imp  OLEQUERYCREATEFROMDATA (OLE2.7)
 0000:0000  Imp  OLEQUERYLINKFROMDATA (OLE2.6)
 0000:0000  Imp  OLESAVE              (OLE2.13)
 0000:0000  Imp  OLESAVETOSTREAM      (OLE2.24)
 0000:0000  Imp  OLESETCONTAINEDOBJECT (OLE2.86)
 0000:0000  Unr  OLESTDCHECKVTBL
 0000:0000  Unr  OLESTDCOMMITSTORAGE
 0001:8842       OLESTDCOMPAREFORMATETC
 0001:8910       OLESTDCOMPARETARGETDEVICE
 0000:0000  Unr  OLESTDCOPYFORMATETC
 0001:771C       OLESTDCOPYSTRING
 0001:87F0       OLESTDCOPYTARGETDEVICE
 0000:0000  Unr  OLESTDCREATECHILDSTORAGE
 0000:0000  Unr  OLESTDCREATEDC
 0000:0000  Unr  OLESTDCREATEIC
 0000:0000  Unr  OLESTDCREATEROOTSTORAGE
 0001:77A6       OLESTDCREATESTORAGEONHGLOBAL
 0000:0000  Unr  OLESTDCREATETARGETDEVICE
 0000:0000  Unr  OLESTDCREATETEMPFILEMONIKER
 0001:783E       OLESTDCREATETEMPSTORAGE
 0000:0000  Unr  OLESTDDELETETARGETDEVICE
 0000:0000  Unr  OLESTDDESTROYALLELEMENTS
 0000:0000  Unr  OLESTDDOCONVERT
 0000:0000  Unr  OLESTDDOTREATASCLASS
 0000:0000  Unr  OLESTDFILLOBJECTDESCRIPTORFROMDATA
 0001:7670       OLESTDFREE
 0001:76C6       OLESTDFREESTRING
 0000:0000  Unr  OLESTDGETAUXUSERTYPE
 0001:7516       OLESTDGETDATA
 0001:8C28       OLESTDGETDEFAULTFILEFORMATOFCLASS
 0001:7AEE       OLESTDGETFIRSTMONIKER
 0000:0000  Unr  OLESTDGETITEMTOKEN
 0000:0000  Unr  OLESTDGETLENFILEPREFIXOFMONIKER
 0000:0000  Unr  OLESTDGETLINKSOURCEDATA
 0000:0000  Unr  OLESTDGETMETAFILEPICTFROMOLEOBJECT
 0000:0000  Unr  OLESTDGETMISCSTATUSOFCLASS
 0001:789C       OLESTDGETOBJECTDESCRIPTORDATA
 0000:0000  Unr  OLESTDGETOBJECTDESCRIPTORDATAFROMOLEOBJECT
 0000:0000  Unr  OLESTDGETOLEOBJECTDATA
 0000:0000  Unr  OLESTDGETPRIORITYCLIPBOARDFORMAT
 0000:0000  Unr  OLESTDGETSIZE
 0000:0000  Unr  OLESTDGETTREATASFMTUSERTYPE
 0001:8AA4       OLESTDGETUSERTYPEOFCLASS
 0000:0000  Unr  OLESTDINITVTBL
 0000:0000  Unr  OLESTDISDUPLICATEFORMAT
 0000:0000  Unr  OLESTDISOLELINK
 0001:7612       OLESTDMALLOC
 0001:7BA4       OLESTDMARKPASTEENTRYLIST
 0000:0000  Unr  OLESTDMKPARSEDISPLAYNAME
 0000:0000  Unr  OLESTDNOTEFILECHANGETIME
 0000:0000  Unr  OLESTDNOTEOBJECTCHANGETIME
 0000:0000  Unr  OLESTDOPENCHILDSTORAGE
 0000:0000  Unr  OLESTDOPENORCREATEROOTSTORAGE
 0000:0000  Unr  OLESTDOPENROOTSTORAGE
 0001:74D8       OLESTDQUERYINTERFACE
 0000:0000  Unr  OLESTDREALLOC
 0000:0000  Unr  OLESTDREGISTERASRUNNING
 0001:7A46       OLESTDRELEASE
 0000:0000  Unr  OLESTDREVOKEASRUNNING
 0000:0000  Unr  OLESTDSETICONINCACHE
 0000:0000  Unr  OLESTDSETUPADVISES
 0000:0000  Unr  OLESTDSWITCHDISPLAYASPECT
 0001:7A22       OLESTDVERIFYRELEASE
 0000:0000  Imp  OLETRANSLATEACCELERATOR (OLE2.78)
 0000:0000  Unr  OLEUIADDVERBMENU
 0000:0000  Unr  OLEUICANUNLOADNOW
 0001:70F4       OLEUIDRAWHANDLES
 0001:7322       OLEUIDRAWSHADING
 0001:64E6       OLEUIINITIALIZE
 0000:0000  Unr  OLEUIMETAFILEPICTEXTRACTICON
 0000:0000  Unr  OLEUIMETAFILEPICTEXTRACTICONSOURCE
 0000:0000  Unr  OLEUIMETAFILEPICTEXTRACTLABEL
 0001:8250       OLEUIMETAFILEPICTICONDRAW
 0001:8208       OLEUIMETAFILEPICTICONFREE
 0000:0000  Unr  OLEUISHOWOBJECT
 0001:666A       OLEUIUNINITIALIZE
 0000:0000  Unr  OLEUIUPDATELINKS
 0000:0000  Imp  OLEUNINITIALIZE      (OLE2.3)
 0000:0000  Imp  OUTPUTDEBUGSTRING    (KERNEL.115)
 0001:6DCA       PARSECMDLINE
 0000:0000  Imp  PATBLT               (GDI.29)
 0000:0000  Imp  PEEKMESSAGE          (USER.109)
 0000:0000  Imp  PLAYMETAFILE         (GDI.123)
 0000:0000  Imp  PLAYMETAFILERECORD   (GDI.176)
 0000:0000  Imp  POSTMESSAGE          (USER.110)
 0000:0000  Imp  POSTQUITMESSAGE      (USER.6)
 0000:0000  Imp  PROGIDFROMCLSID      (COMPOBJ.62)
 0001:6682       PROMPTUSERDLGPROC
 0000:0000  Imp  READCLASSSTG         (OLE2.18)
 0000:0000  Imp  READFMTUSERTYPESTG   (OLE2.74)
 0000:0000  Imp  RECTANGLE            (GDI.27)
 0000:0000  Imp  REGCLOSEKEY          (SHELL.3)
 0000:0000  Imp  REGISTERCLASS        (USER.57)
 0000:0000  Imp  REGISTERCLIPBOARDFORMAT (USER.145)
 0001:615E       REGISTERHATCHWINDOWCLASS
 0000:0000  Imp  REGISTERWINDOWMESSAGE (USER.118)
 0000:0000  Imp  REGOPENKEY           (SHELL.1)
 0000:0000  Imp  REGQUERYVALUE        (SHELL.6)
 0000:0000  Imp  REGSETVALUE          (SHELL.5)
 0000:0000  Imp  RELEASEDC            (USER.68)
 0000:0000  Imp  RELEASESTGMEDIUM     (OLE2.32)
 0000:0000  Imp  REMOVEMENU           (USER.412)
 0000:0000  Imp  REMOVEPROP           (USER.24)
 0000:0000  Unr  RESETORIGDC
 0000:0000  Imp  RESTOREDC            (GDI.39)
 0001:7F0E       RESULTIMAGEWNDPROC
 0002:0004       rsrvptrs
 0000:0000  Imp  SAVEDC               (GDI.30)
 0000:0000  Imp  SELECTOBJECT         (GDI.45)
 0000:0000  Imp  SENDMESSAGE          (USER.111)
 0000:0000  Imp  SETBKCOLOR           (GDI.1)
 0000:0000  Imp  SETBKMODE            (GDI.2)
 0000:0000  Imp  SETBRUSHORG          (GDI.148)
 0000:0000  Imp  SETCONVERTSTG        (OLE2.83)
 0000:0000  Imp  SETCURSOR            (USER.69)
 0000:0000  Unr  SETDCTOANISOTROPIC
 0000:0000  Unr  SETDCTODRAWINHIMETRICRECT
 0000:0000  Imp  SETDIBITS            (GDI.440)
 0000:0000  Imp  SETDLGITEMTEXT       (USER.92)
 0000:0000  Imp  SETFOCUS             (USER.22)
 0001:62A6       SETHATCHRECT
 0001:630A       SETHATCHWINDOWSIZE
 0000:0000  Imp  SETMAPMODE           (GDI.3)
 0000:0000  Imp  SETMESSAGEQUEUE      (USER.266)
 0000:0000  Imp  SETPARENT            (USER.233)
 0000:0000  Imp  SETPROP              (USER.26)
 0000:0000  Imp  SETRECT              (USER.72)
 0000:0000  Imp  SETRECTEMPTY         (USER.73)
 0000:0000  Imp  SETTEXTCOLOR         (GDI.9)
 0000:0000  Imp  SETTIMER             (USER.10)
 0000:0000  Imp  SETVIEWPORTEXT       (GDI.14)
 0000:0000  Imp  SETVIEWPORTEXTEX     (GDI.479)
 0000:0000  Imp  SETVIEWPORTORGEX     (GDI.480)
 0000:0000  Imp  SETWINDOWEXT         (GDI.12)
 0000:0000  Imp  SETWINDOWEXTEX       (GDI.481)
 0000:0000  Imp  SETWINDOWORG         (GDI.11)
 0000:0000  Imp  SETWINDOWORGEX       (GDI.482)
 0000:0000  Imp  SETWINDOWTEXT        (USER.37)
 0000:0000  Imp  SETWINDOWWORD        (USER.134)
 0000:0000  Imp  SHOWWINDOW           (USER.42)
 0000:0000  Imp  STGCREATEDOCFILE     (STORAGE.1)
 0000:0000  Imp  STGCREATEDOCFILEONILOCKBYTES (STORAGE.2)
 0000:0000  Imp  STGOPENSTORAGE       (STORAGE.3)
 0000:0000  Imp  STRINGFROMCLSID      (COMPOBJ.19)
 0000:0000  Imp  TRANSLATEMESSAGE     (USER.113)
 0000:0000  Imp  UNREALIZEOBJECT      (GDI.150)
 0001:6728       UPDATELINKSDLGPROC
 0000:0000  Imp  UPDATEWINDOW         (USER.124)
 0000:0000  Imp  WAITEVENT            (KERNEL.30)
 0001:38B6       WINMAIN
 0000:0000  Imp  WRITECLASSSTG        (OLE2.19)
 0000:0000  Imp  WRITECLASSSTM        (OLE2.21)
 0000:0000  Imp  WRITEFMTUSERTYPESTG  (OLE2.75)
 0000:0000  Imp  WVSPRINTF            (USER.421)
 0001:6CCE       XFORMHEIGHTINHIMETRICTOPIXELS
 0001:6C82       XFORMHEIGHTINPIXELSTOHIMETRIC
 0000:0000  Unr  XFORMRECTINHIMETRICTOPIXELS
 0001:6D1A       XFORMRECTINPIXELSTOHIMETRIC
 0000:0000  Unr  XFORMSIZEINHIMETRICTOPIXELS
 0000:0000  Unr  XFORMSIZEINPIXELSTOHIMETRIC
 0001:6C36       XFORMWIDTHINHIMETRICTOPIXELS
 0001:6BEA       XFORMWIDTHINPIXELSTOHIMETRIC
 0001:3D0C       _abs
 0002:0E5E       _aseghi
 0002:0E5C       _aseglo
 0001:4E8A       _atof
 0002:1F32       _cfEmbeddedObject
 0002:1F30       _cfEmbedSource
 0002:1F3A       _cfFileName
 0002:1F3C       _cfLinkSource
 0002:1F38       _cfLinkSrcDescriptor
 0002:1F46       _cfObjectDescriptor
 0002:1F36       _cfOwnerLink
 0002:14E2       _edata
 0002:1F48       _end
 0002:0F96       _errno
 0001:4047       _exit
 0001:6EF2       _FIconBoxInitialize
 0001:7E0C       _FResultImageInitialize
 0002:1F34       _ghInst
 0000:0000  Imp  _GUID_NULL           (COMPOBJ.37)
 0001:005D       _GUID_SIMPLE
 0002:0E14       _g_dwLockCount
 0002:0E10       _g_dwObjectCount
 0001:6F68       _IconBoxUninitialize
 0000:0000  Imp  _IID_IClassFactory   (COMPOBJ.39)
 0000:0000  Imp  _IID_IDataObject     (OLE2.134)
 0000:0000  Imp  _IID_IExternalConnection (COMPOBJ.72)
 0000:0000  Imp  _IID_IOleCache       (OLE2.150)
 0000:0000  Imp  _IID_IOleInPlaceActiveObject (OLE2.143)
 0000:0000  Imp  _IID_IOleInPlaceObject (OLE2.139)
 0000:0000  Imp  _IID_IOleInPlaceSite (OLE2.145)
 0000:0000  Imp  _IID_IOleLink        (OLE2.149)
 0000:0000  Imp  _IID_IOleObject      (OLE2.138)
 0000:0000  Imp  _IID_IPersist        (OLE2.132)
 0000:0000  Imp  _IID_IPersistStorage (OLE2.130)
 0000:0000  Imp  _IID_IUnknown        (COMPOBJ.38)
 0000:0000  Imp  _IID_IViewObject     (OLE2.133)
 0000:0000  Imp  _IID_IViewObject2    (OLE2.158)
 0001:7A6A       _OleStdNullMethod
 0000:0000  Unr  _OleUIPromptUser
 0001:7EFC       _ResultImageUninitialize
 0002:0E50       _STKHQQ
 0001:518A       _strlen
 0001:389E       _TestDebugOut
 0001:807E       _TransparentBlt
 0002:0E1C       _uMsgBrowse
 0002:0E1E       _uMsgChangeIcon
 0002:0E22       _uMsgCloseBusyDlg
 0002:0E1A       _uMsgEndDialog
 0002:0E20       _uMsgFileOKString
 0002:0E18       _uMsgHelp
 0000:0000  Imp  _wsprintf            (USER.420)
 0002:0F7A       __acfinfo
 0000:9876  Abs  __acrtmsg
 0000:9876  Abs  __acrtused
 0000:D6D6  Abs  __aDBdoswp
 0002:0FE8       __adbgmsg
 0000:D6D6  Abs  __aDBused
 0001:51A4       __aFahdiff
 0001:3EE6       __aFftol
 0001:3DB2       __aFlmul
 0001:3DB2       __aFulmul
 0000:0000  Imp  __AHINCR             (KERNEL.114)
 0000:0000  Imp  __AHSHIFT            (KERNEL.113)
 0002:0F88       __aintdiv
 0002:1046       __amblksiz
 0001:43B4       __amsg_exit
 0002:1028       __asizeC
 0002:1029       __asizeD
 0001:3C2C       __astart
 0001:4064       __cexit
 0001:4AEA       __cfltcvt
 0002:1008       __cfltcvt_tab
 0001:46A6       __cftoe
 0001:4872       __cftof
 0001:4A0A       __cftog
 0002:0FE5       __child
 0001:3F64       __cinit
 0001:43AA       __cintDIV
 0002:0E5A       __cmdShow
 0002:0FA5       __cpumode
 0001:4592       __cropzeros
 0001:40E5       __ctermsub
 0002:0E64       __ctype
 0002:0E64       __ctype_
 0001:4075       __c_exit
 0002:0FA6       __doserrno
 0001:43F6       __dosret0
 0001:4415       __dosretax
 0001:4403       __dosreturn
 0001:3D38       __dos_findfirst
 0001:3D26       __dos_findnext
 0002:14E2       __edata
 0002:1F48       __end
 0002:0FDC       __environ
 0001:4055       __exit
 0002:0FE7       __exitflag
 0002:0F8C       __fac
 0001:464E       __fassign
 0001:4454       __ffree
 0001:4122       __FF_MSGBANNER
 0002:1038       __fheap
 0001:4DE7       __findlast
 0001:5358       __fltin
 0001:50B6       __fltout
 0000:9876  Abs  __fltused
 0001:4475       __fmalloc
 0001:3DE4       __fmemcmp
 0001:3E40       __fmemcpy
 0001:4FEC       __fmemmove
 0001:3E9E       __fmemset
 0001:451C       __forcdecpt
 0002:10C4       __fpinit
 0000:0000  Imp  __fpmath             (WIN87EM.1)
 0001:4B8C       __fpsignal
 0000:9876  Abs  __fptaskdata
 0001:4EE8       __fptostr
 0001:4BBC       __fptrap
 0001:3D20       __fpurecall
 0001:4FB0       __fstrcpy
 0001:4F96       __fstrlen
 0001:3EE6       __ftol
 0001:4C64       __GetDGROUP
 0001:4CF0       __growseg
 0002:0E54       __hInstance
 0002:0E52       __hPrevInstance
 0001:4D81       __incseg
 0001:5120       __initseg
 0001:5BD3       __LD12MULT
 0001:5AFE       __LD12MULTTENPOWER
 0001:5154       __linkseg
 0002:0E56       __lpszCmdLine
 0001:5D58       __MANTOLD12
 0001:4427       __maperror
 0002:1F3E       __mbac
 0001:4C36       __myalloc
 0001:4E08       __newseg
 0002:0FA8       __nfile
 0001:4BC2       __NMSG_TEXT
 0001:4BF9       __NMSG_WRITE
 0001:3CE3       __nomain
 0001:3D20       __npurecall
 0002:0FA6       __oserr
 0002:0FAE       __osfile
 0002:0FA1       __osmajor
 0002:0FA0       __osminor
 0002:0FA4       __osmode
 0002:0FA0       __osver
 0002:0FA2       __osversion
 0002:0FE0       __pgmptr
 0002:1004       __pnhFarHeap
 0001:4616       __positive
 0002:0F9C       __psp
 0002:0F9A       __pspadr
 0001:3D20       __purecall
 0001:4BB5       __QWINClose
 0001:4BB5       __QWINExit
 0001:4BB5       __QWINGetBuffSize
 0001:4BB5       __QWINGetFocus
 0001:4BB5       __QWINGetSize
 0001:4BB5       __QWINInit
 0001:4BB5       __QWINIsQWINin
 0001:4BB5       __QWINMenuClick
 0001:4BB5       __QWINOpen
 0001:4BB5       __QWINRead
 0001:4BB5       __QWINSetAboutString
 0001:4BB5       __QWINSetBuffSize
 0001:4BB5       __QWINSetFocus
 0001:4BB5       __QWINSetSize
 0001:4BB5       __QWINTerm
 0002:1036       __qwinused
 0001:4BB5       __QWINWrite
 0001:4BB5       __QWINYield
 0001:4C74       __searchseg
 0001:4146       __setargv
 0001:42F0       __setenvp
 0002:1026       __sigintoff
 0002:1024       __sigintseg
 0000:0001  Abs  __sizec
 0000:0001  Abs  __sized
 0001:5576       __STRINGTOD
 0001:55DE       __STRINGTOLD
 0001:3F38       __stubmain
 0002:0F98       __umaskval
 0001:4BB5       __wabout
 0001:4BB0       __wcexit
 0001:4BB0       __wcinit
 0001:4BB5       __wclose
 0002:0FAA       __wfile
 0001:3C22       __wflags
 0001:4BB5       __wgetfocus
 0001:4BB5       __wgetscreenbuf
 0001:4BB5       __wgetsize
 0000:0000  Imp  __WINFLAGS           (KERNEL.178)
 0002:0F9F       __winmajor
 0002:0F9E       __winminor
 0002:0F9E       __winver
 0000:0000  Abs  __wiobused
 0001:4BB5       __wmenuclick
 0002:0FAC       __wnfile
 0001:4BB5       __wopen
 0001:4BB5       __wread
 0001:4BB5       __wsetfocus
 0001:4BB5       __wsetscreenbuf
 0001:4BB5       __wsetsize
 0002:0FC2       __wsfile
 0001:4BB5       __wterm
 0001:4BB5       __wwrite
 0002:0E62       ___aDBrterr
 0002:0E60       ___aDBswpflg
 0002:0FD6       ___argc
 0002:0FD8       ___argv
 0001:510C       ___ExportedStub

  Address         Publics by Value

 0000:0000  Imp  OFFSETRECT           (USER.77)
 0000:0000  Imp  FINDRESOURCE         (KERNEL.60)
 0000:0000  Imp  GETCLASSFILE         (OLE2.57)
 0000:0000  Unr  XFORMRECTINHIMETRICTOPIXELS
 0000:0000  Imp  CREATEMENU           (USER.151)
 0000:0000  Imp  CREATEIC             (GDI.153)
 0000:0000  Imp  CREATEDC             (GDI.53)
 0000:0000  Imp  LOADBITMAP           (USER.175)
 0000:0000  Imp  RELEASEDC            (USER.68)
 0000:0000  Imp  SETBRUSHORG          (GDI.148)
 0000:0000  Unr  OLESTDCREATETEMPFILEMONIKER
 0000:0000  Unr  OLESTDGETMISCSTATUSOFCLASS
 0000:0000  Unr  OLESTDDOTREATASCLASS
 0000:0000  Imp  REGISTERCLIPBOARDFORMAT (USER.145)
 0000:0000  Imp  RELEASESTGMEDIUM     (OLE2.32)
 0000:0000  Imp  SETWINDOWTEXT        (USER.37)
 0000:0000  Imp  PROGIDFROMCLSID      (COMPOBJ.62)
 0000:0000  Imp  REGISTERWINDOWMESSAGE (USER.118)
 0000:0000  Imp  GLOBALFREE           (KERNEL.17)
 0000:0000  Imp  SETWINDOWORGEX       (GDI.482)
 0000:0000  Imp  MKPARSEDISPLAYNAME   (OLE2.23)
 0000:0000  Unr  OLEUIMETAFILEPICTEXTRACTICON
 0000:0000  Unr  OLESTDOPENCHILDSTORAGE
 0000:0000  Unr  RESETORIGDC
 0000:0000  Imp  DESTROYMENU          (USER.152)
 0000:0000  Imp  UPDATEWINDOW         (USER.124)
 0000:0000  Imp  _IID_IUnknown        (COMPOBJ.38)
 0000:0000  Imp  ISWINDOW             (USER.47)
 0000:0000  Unr  OLEUIMETAFILEPICTEXTRACTICONSOURCE
 0000:0000  Imp  SETMAPMODE           (GDI.3)
 0000:0000  Unr  OLESTDGETOBJECTDESCRIPTORDATAFROMOLEOBJECT
 0000:0000  Imp  CREATEICON           (USER.407)
 0000:0000  Imp  STGOPENSTORAGE       (STORAGE.3)
 0000:0000  Imp  WRITEFMTUSERTYPESTG  (OLE2.75)
 0000:0000  Imp  UNREALIZEOBJECT      (GDI.150)
 0000:0000  Imp  LOADRESOURCE         (KERNEL.61)
 0000:0000  Unr  OLESTDCREATEDC
 0000:0000  Unr  OLESTDCREATEIC
 0000:0000  Imp  INSERTMENU           (USER.410)
 0000:0000  Imp  GETPARENT            (USER.46)
 0000:0000  Imp  ISBADREADPTR         (KERNEL.334)
 0000:0000  Imp  FATALEXIT            (KERNEL.1)
 0000:0000  Unr  OLESTDGETPRIORITYCLIPBOARDFORMAT
 0000:0000  Unr  OLESTDGETLINKSOURCEDATA
 0000:0000  Imp  CREATECOMPATIBLEBITMAP (GDI.51)
 0000:0000  Imp  OLEDUPLICATEDATA     (OLE2.51)
 0000:0000  Imp  POSTQUITMESSAGE      (USER.6)
 0000:0000  Imp  COPYRECT             (USER.74)
 0000:0000  Imp  LOCKRESOURCE         (KERNEL.62)
 0000:0000  Imp  CREATEBINDCTX        (OLE2.26)
 0000:0000  Imp  DISPATCHMESSAGE      (USER.114)
 0000:0000  Imp  DELETEMETAFILE       (GDI.127)
 0000:0000  Imp  DOS3CALL             (KERNEL.102)
 0000:0000  Unr  XFORMSIZEINPIXELSTOHIMETRIC
 0000:0000  Imp  SETDIBITS            (GDI.440)
 0000:0000  Imp  READCLASSSTG         (OLE2.18)
 0000:0000  Imp  GETSYSTEMMETRICS     (USER.179)
 0000:0000  Imp  INVERTRECT           (USER.82)
 0000:0000  Imp  FREEPROCINSTANCE     (KERNEL.52)
 0000:0000  Imp  REGISTERCLASS        (USER.57)
 0000:0000  Unr  OLESTDGETLENFILEPREFIXOFMONIKER
 0000:0000  Imp  LOADICON             (USER.174)
 0000:0000  Imp  _IID_IClassFactory   (COMPOBJ.39)
 0000:0000  Imp  ENDPAINT             (USER.40)
 0000:0000  Imp  __WINFLAGS           (KERNEL.178)
 0000:0000  Unr  OLESTDOPENORCREATEROOTSTORAGE
 0000:0000  Unr  OLESTDCOMMITSTORAGE
 0000:0000  Unr  OLESTDCREATETARGETDEVICE
 0000:0000  Imp  FREERESOURCE         (KERNEL.63)
 0000:0000  Imp  WVSPRINTF            (USER.421)
 0000:0000  Imp  CREATEFILEMONIKER    (OLE2.28)
 0000:0000  Imp  GETPROP              (USER.25)
 0000:0000  Imp  SETPROP              (USER.26)
 0000:0000  Imp  STGCREATEDOCFILEONILOCKBYTES (STORAGE.2)
 0000:0000  Unr  OLESTDDELETETARGETDEVICE
 0000:0000  Imp  GETDLGITEM           (USER.91)
 0000:0000  Imp  SETBKCOLOR           (GDI.1)
 0000:0000  Unr  OLESTDFILLOBJECTDESCRIPTORFROMDATA
 0000:0000  Imp  SETDLGITEMTEXT       (USER.92)
 0000:0000  Imp  GETDLGITEMTEXT       (USER.93)
 0000:0000  Imp  OLECREATEMENUDESCRIPTOR (OLE2.40)
 0000:0000  Imp  GETBKCOLOR           (GDI.75)
 0000:0000  Imp  _IID_IViewObject2    (OLE2.158)
 0000:0000  Imp  SETWINDOWEXT         (GDI.12)
 0000:0000  Imp  RESTOREDC            (GDI.39)
 0000:0000  Imp  PLAYMETAFILERECORD   (GDI.176)
 0000:0000  Unr  OLEUICANUNLOADNOW
 0000:0000  Imp  CLSIDFROMPROGID      (COMPOBJ.61)
 0000:0000  Imp  SETCURSOR            (USER.69)
 0000:0000  Imp  SETBKMODE            (GDI.2)
 0000:0000  Imp  LOADCURSOR           (USER.173)
 0000:0000  Imp  ENDDIALOG            (USER.88)
 0000:0000  Imp  CREATEDATAADVISEHOLDER (OLE2.39)
 0000:0000  Imp  BITBLT               (GDI.34)
 0000:0000  Unr  OLEUISHOWOBJECT
 0000:0000  Imp  FRAMERECT            (USER.83)
 0000:0000  Unr  OLESTDDOCONVERT
 0000:0000  Imp  SETTIMER             (USER.10)
 0000:0000  Unr  OLESTDISDUPLICATEFORMAT
 0000:0000  Imp  LSTRCPYN             (KERNEL.353)
 0000:0000  Imp  SENDMESSAGE          (USER.111)
 0000:0000  Imp  __fpmath             (WIN87EM.1)
 0000:0000  Imp  REMOVEPROP           (USER.24)
 0000:0000  Imp  OLESAVE              (OLE2.13)
 0000:0000  Imp  COGETMALLOC          (COMPOBJ.4)
 0000:0000  Unr  OLESTDNOTEFILECHANGETIME
 0000:0000  Imp  GETSUBMENU           (USER.159)
 0000:0000  Unr  OLESTDGETTREATASFMTUSERTYPE
 0000:0000  Imp  _IID_IOleObject      (OLE2.138)
 0000:0000  Imp  REGOPENKEY           (SHELL.1)
 0000:0000  Imp  __AHSHIFT            (KERNEL.113)
 0000:0000  Imp  MOVEWINDOW           (USER.56)
 0000:0000  Imp  PEEKMESSAGE          (USER.109)
 0000:0000  Imp  SETRECTEMPTY         (USER.73)
 0000:0000  Imp  STGCREATEDOCFILE     (STORAGE.1)
 0000:0000  Imp  OLESAVETOSTREAM      (OLE2.24)
 0000:0000  Imp  SELECTOBJECT         (GDI.45)
 0000:0000  Unr  OLESTDNOTEOBJECTCHANGETIME
 0000:0000  Imp  FILLRECT             (USER.81)
 0000:0000  Imp  SETVIEWPORTEXT       (GDI.14)
 0000:0000  Imp  DIALOGBOXPARAM       (USER.239)
 0000:0000  Imp  _IID_IPersist        (OLE2.132)
 0000:0000  Imp  GETWINDOWWORD        (USER.133)
 0000:0000  Imp  SETWINDOWWORD        (USER.134)
 0000:0000  Imp  _IID_IExternalConnection (COMPOBJ.72)
 0000:0000  Imp  COREGISTERCLASSOBJECT (COMPOBJ.5)
 0000:0000  Imp  CREATEPATTERNBRUSH   (GDI.60)
 0000:0000  Imp  GLOBALUNLOCK         (KERNEL.19)
 0000:0000  Imp  CODISCONNECTOBJECT   (COMPOBJ.15)
 0000:0000  Unr  OLESTDCREATEROOTSTORAGE
 0000:0000  Imp  CREATESOLIDBRUSH     (GDI.66)
 0000:0000  Imp  GLOBALLOCK           (KERNEL.18)
 0000:0000  Imp  SETWINDOWEXTEX       (GDI.481)
 0000:0000  Imp  _IID_IOleInPlaceSite (OLE2.145)
 0000:0000  Imp  REMOVEMENU           (USER.412)
 0000:0000  Imp  GETDEVICECAPS        (GDI.80)
 0000:0000  Imp  OLEBUILDVERSION      (OLE2.1)
 0000:0000  Imp  COREVOKECLASSOBJECT  (COMPOBJ.6)
 0000:0000  Imp  _GUID_NULL           (COMPOBJ.37)
 0000:0000  Imp  REGSETVALUE          (SHELL.5)
 0000:0000  Unr  OLEUIADDVERBMENU
 0000:0000  Imp  _IID_IOleInPlaceObject (OLE2.139)
 0000:0000  Imp  GETRUNNINGOBJECTTABLE (OLE2.30)
 0000:0000  Imp  CREATECOMPATIBLEDC   (GDI.52)
 0000:0000  Imp  DESTROYWINDOW        (USER.53)
 0000:0000  Unr  OLESTDOPENROOTSTORAGE
 0000:0000  Imp  LSTRLEN              (KERNEL.90)
 0000:0000  Unr  OLESTDSETUPADVISES
 0000:0000  Imp  SETCONVERTSTG        (OLE2.83)
 0000:0000  Imp  OLETRANSLATEACCELERATOR (OLE2.78)
 0000:0000  Imp  DELETEOBJECT         (GDI.69)
 0000:0000  Imp  _wsprintf            (USER.420)
 0000:0000  Unr  SETDCTODRAWINHIMETRICRECT
 0000:0000  Imp  SETFOCUS             (USER.22)
 0000:0000  Imp  _IID_IViewObject     (OLE2.133)
 0000:0000  Imp  WAITEVENT            (KERNEL.30)
 0000:0000  Imp  ANSINEXT             (USER.472)
 0000:0000  Imp  DELETEDC             (GDI.68)
 0000:0000  Unr  OLEUIMETAFILEPICTEXTRACTLABEL
 0000:0000  Imp  COFILETIMENOW        (COMPOBJ.82)
 0000:0000  Unr  OLESTDCOPYFORMATETC
 0000:0000  Imp  CODOSDATETIMETOFILETIME (COMPOBJ.31)
 0000:0000  Imp  GETCLIENTRECT        (USER.33)
 0000:0000  Imp  INVALIDATERECT       (USER.125)
 0000:0000  Imp  _IID_IOleCache       (OLE2.150)
 0000:0000  Imp  CREATEBRUSHINDIRECT  (GDI.50)
 0000:0000  Imp  SETTEXTCOLOR         (GDI.9)
 0000:0000  Imp  MULDIV               (GDI.128)
 0000:0000  Imp  TRANSLATEMESSAGE     (USER.113)
 0000:0000  Imp  INITAPP              (USER.5)
 0000:0000  Imp  FATALAPPEXIT         (KERNEL.137)
 0000:0000  Imp  LOCKSEGMENT          (KERNEL.23)
 0000:0000  Unr  OLESTDGETITEMTOKEN
 0000:0000  Unr  OLESTDISOLELINK
 0000:0000  Imp  _IID_IOleLink        (OLE2.149)
 0000:0000  Unr  OLESTDREVOKEASRUNNING
 0000:0000  Imp  GETSTOCKOBJECT       (GDI.87)
 0000:0000  Imp  __AHINCR             (KERNEL.114)
 0000:0000  Unr  OLEUIUPDATELINKS
 0000:0000  Unr  XFORMSIZEINHIMETRICTOPIXELS
 0000:0000  Imp  LSTRCMP              (USER.430)
 0000:0000  Imp  LSTRCAT              (KERNEL.89)
 0000:0000  Unr  _OleUIPromptUser
 0000:0000  Imp  ISDBCSLEADBYTE       (KERNEL.207)
 0000:0000  Imp  READFMTUSERTYPESTG   (OLE2.74)
 0000:0000  Imp  LSTRCPY              (KERNEL.88)
 0000:0000  Imp  GLOBALALLOC          (KERNEL.15)
 0000:0000  Imp  OUTPUTDEBUGSTRING    (KERNEL.115)
 0000:0000  Imp  MESSAGEBOX           (USER.1)
 0000:0000  Unr  OLESTDSWITCHDISPLAYASPECT
 0000:0000  Imp  ANSITOOEM            (KEYBOARD.5)
 0000:0000  Imp  _IID_IPersistStorage (OLE2.130)
 0000:0000  Imp  SETRECT              (USER.72)
 0000:0000  Imp  CREATESTREAMONHGLOBAL (OLE2.84)
 0000:0000  Imp  GLOBALREALLOC        (KERNEL.16)
 0000:0000  Unr  OLESTDGETSIZE
 0000:0000  Imp  SETVIEWPORTEXTEX     (GDI.479)
 0000:0000  Imp  SAVEDC               (GDI.30)
 0000:0000  Imp  GETOBJECT            (GDI.82)
 0000:0000  Imp  GETMENU              (USER.157)
 0000:0000  Imp  PATBLT               (GDI.29)
 0000:0000  Imp  ISDIALOGMESSAGE      (USER.90)
 0000:0000  Unr  OLESTDGETAUXUSERTYPE
 0000:0000  Imp  INITTASK             (KERNEL.91)
 0000:0000  Unr  OLESTDCREATECHILDSTORAGE
 0000:0000  Imp  CREATEOLEADVISEHOLDER (OLE2.38)
 0000:0000  Imp  GETVERSION           (KERNEL.3)
 0000:0000  Imp  OLEQUERYCREATEFROMDATA (OLE2.7)
 0000:0000  Imp  GETDC                (USER.66)
 0000:0000  Imp  INFLATERECT          (USER.78)
 0000:0000  Imp  OLEDESTROYMENUDESCRIPTOR (OLE2.42)
 0000:0000  Imp  SETVIEWPORTORGEX     (GDI.480)
 0000:0000  Unr  OLESTDGETOLEOBJECTDATA
 0000:0000  Imp  OLEUNINITIALIZE      (OLE2.3)
 0000:0000  Imp  STRINGFROMCLSID      (COMPOBJ.19)
 0000:0000  Imp  CREATEILOCKBYTESONHGLOBAL (OLE2.54)
 0000:0000  Imp  GETDOSENVIRONMENT    (KERNEL.131)
 0000:0000  Imp  CREATEWINDOW         (USER.41)
 0000:0000  Imp  GLOBALSIZE           (KERNEL.20)
 0000:0000  Imp  ISEQUALGUID          (COMPOBJ.18)
 0000:0000  Imp  RECTANGLE            (GDI.27)
 0000:0000  Imp  CLOSEMETAFILE        (GDI.126)
 0000:0000  Imp  OLESETCONTAINEDOBJECT (OLE2.86)
 0000:0000  Unr  OLESTDCHECKVTBL
 0000:0000  Imp  GETPROFILEINT        (KERNEL.57)
 0000:0000  Imp  GETBITMAPBITS        (GDI.74)
 0000:0000  Imp  GETMODULEFILENAME    (KERNEL.49)
 0000:0000  Imp  DIALOGBOX            (USER.87)
 0000:0000  Imp  COTREATASCLASS       (COMPOBJ.66)
 0000:0000  Imp  MAKEPROCINSTANCE     (KERNEL.51)
 0000:0000  Unr  OLESTDINITVTBL
 0000:0000  Imp  GETMESSAGE           (USER.108)
 0000:0000  Unr  OLESTDDESTROYALLELEMENTS
 0000:0000  Unr  OLESTDGETMETAFILEPICTFROMOLEOBJECT
 0000:0000  Imp  SETWINDOWORG         (GDI.11)
 0000:0000  Imp  CREATEPEN            (GDI.61)
 0000:0000  Imp  DELETEMENU           (USER.413)
 0000:0000  Unr  OLESTDMKPARSEDISPLAYNAME
 0000:0000  Unr  OLESTDSETICONINCACHE
 0000:0000  Imp  INTERSECTRECT        (USER.79)
 0000:0000  Imp  KILLTIMER            (USER.12)
 0000:0000  Imp  OLEQUERYLINKFROMDATA (OLE2.6)
 0000:0000  Imp  SHOWWINDOW           (USER.42)
 0000:0000  Imp  LOADSTRING           (USER.176)
 0000:0000  Imp  SETPARENT            (USER.233)
 0000:0000  Imp  CREATEMETAFILE       (GDI.125)
 0000:0000  Unr  OLESTDREALLOC
 0000:0000  Imp  SETMESSAGEQUEUE      (USER.266)
 0000:0000  Imp  CREATEPOPUPMENU      (USER.415)
 0000:0000  Imp  REGQUERYVALUE        (SHELL.6)
 0000:0000  Imp  GETSYSCOLOR          (USER.180)
 0000:0000  Imp  POSTMESSAGE          (USER.110)
 0000:0000  Imp  ENUMMETAFILE         (GDI.175)
 0000:0000  Imp  LSTRCMPI             (USER.471)
 0000:0000  Abs  __wiobused
 0000:0000  Imp  PLAYMETAFILE         (GDI.123)
 0000:0000  Imp  DEFWINDOWPROC        (USER.107)
 0000:0000  Imp  _IID_IOleInPlaceActiveObject (OLE2.143)
 0000:0000  Imp  COLOCKOBJECTEXTERNAL (COMPOBJ.63)
 0000:0000  Imp  WRITECLASSSTM        (OLE2.21)
 0000:0000  Imp  COISOLE1CLASS        (COMPOBJ.36)
 0000:0000  Imp  WRITECLASSSTG        (OLE2.19)
 0000:0000  Imp  _IID_IDataObject     (OLE2.134)
 0000:0000  Imp  REGCLOSEKEY          (SHELL.3)
 0000:0000  Imp  BEGINPAINT           (USER.39)
 0000:0000  Unr  SETDCTOANISOTROPIC
 0000:0000  Unr  OLESTDREGISTERASRUNNING
 0000:0000  Imp  OLEINITIALIZE        (OLE2.2)
 0000:0000  Imp  CREATEBITMAP         (GDI.48)
 0000:0001  Abs  __sized
 0000:0001  Abs  __sizec
 0000:0632  Abs  FISRQQ
 0000:0E32  Abs  FICRQQ
 0000:1632  Abs  FIERQQ
 0000:9876  Abs  __acrtused
 0000:9876  Abs  __fltused
 0000:9876  Abs  __acrtmsg
 0000:9876  Abs  __fptaskdata
 0000:D6D6  Abs  __aDBused
 0000:D6D6  Abs  __aDBdoswp
 0001:0000       ??0CSimpSvrApp@@REC@XZ
 0001:005D       _GUID_SIMPLE
 0001:006E       ??1CSimpSvrApp@@REC@XZ
 0001:00AC       ?QueryInterface@CSimpSvrApp@@VEAPEXAFUGUID@@PEPEX@Z
 0001:0138       ?AddRef@CSimpSvrApp@@VEAKXZ
 0001:015C       ?Release@CSimpSvrApp@@VEAKXZ
 0001:01A8       ?fInitApplication@CSimpSvrApp@@RECHI@Z
 0001:0274       ?fInitInstance@CSimpSvrApp@@RECHIHPEUCClassFactory@@@Z
 0001:0432       ?lCommandHandler@CSimpSvrApp@@RECJIIIJ@Z
 0001:05B4       ?lSizeHandler@CSimpSvrApp@@RECJIIIJ@Z
 0001:05E2       ?lCreateDoc@CSimpSvrApp@@RECJIIIJ@Z
 0001:0618       ?PaintApp@CSimpSvrApp@@RECXI@Z
 0001:063C       ?ParseCmdLine@CSimpSvrApp@@RECXPED@Z
 0001:0664       ?SetStatusText@CSimpSvrApp@@RECXXZ
 0001:067C       ?IsInPlaceActive@CSimpSvrApp@@RECHXZ
 0001:06BA       ?ShowAppWnd@CSimpSvrApp@@RECXH@Z
 0001:06EC       ?HideAppWnd@CSimpSvrApp@@RECXXZ
 0001:0710       ?Create@CSimpSvrDoc@@TAPEV1@PEVCSimpSvrApp@@PEUtagRECT@@I@Z
 0001:07DC       ??0CSimpSvrDoc@@REC@PEVCSimpSvrApp@@I@Z
 0001:0832       ??1CSimpSvrDoc@@REC@XZ
 0001:0872       ?QueryInterface@CSimpSvrDoc@@VEAPEXAFUGUID@@PEPEX@Z
 0001:08E0       ?AddRef@CSimpSvrDoc@@VEAKXZ
 0001:091C       ?Release@CSimpSvrDoc@@VEAKXZ
 0001:0980       ?lResizeDoc@CSimpSvrDoc@@RECJPEUtagRECT@@@Z
 0001:09AA       ?PaintDoc@CSimpSvrDoc@@RECXI@Z
 0001:09F0       ?CreateObject@CSimpSvrDoc@@RECPEXAFUGUID@@PEPEX@Z
 0001:0A78       ?Close@CSimpSvrDoc@@RECXXZ
 0001:0DA0       ?SetStatusText@CSimpSvrDoc@@RECXXZ
 0001:0DE4       ?ShowDocWnd@CSimpSvrDoc@@RECXXZ
 0001:0E06       ?ShowHatchWnd@CSimpSvrDoc@@RECXXZ
 0001:0E1C       ?HideDocWnd@CSimpSvrDoc@@RECXXZ
 0001:0E32       ?HideHatchWnd@CSimpSvrDoc@@RECXXZ
 0001:0E48       ?QueryInterface@CClassFactory@@VEAPEXAFUGUID@@PEPEX@Z
 0001:0EEE       ?AddRef@CClassFactory@@VEAKXZ
 0001:0F12       ?Release@CClassFactory@@VEAKXZ
 0001:0F76       ?CreateInstance@CClassFactory@@VEAPEXPEUIUnknown@@AFUGUID@@PEPEX@Z
 0001:0FDA       ?LockServer@CClassFactory@@VEAPEXH@Z
 0001:100A       ?QueryInterface@CDataObject@@VEAPEXAFUGUID@@PEPEX@Z
 0001:1046       ?AddRef@CDataObject@@VEAKXZ
 0001:107A       ?Release@CDataObject@@VEAKXZ
 0001:10AE       ?QueryGetData@CDataObject@@VEAPEXPEUtagFORMATETC@@@Z
 0001:1108       ?DAdvise@CDataObject@@VEAPEXPEUtagFORMATETC@@KPEUIAdviseSink@@PEK@Z
 0001:1172       ?GetData@CDataObject@@VEAPEXPEUtagFORMATETC@@PEUtagSTGMEDIUM@@@Z
 0001:11F4       ?DUnadvise@CDataObject@@VEAPEXK@Z
 0001:1252       ?GetDataHere@CDataObject@@VEAPEXPEUtagFORMATETC@@PEUtagSTGMEDIUM@@@Z
 0001:1270       ?GetCanonicalFormatEtc@CDataObject@@VEAPEXPEUtagFORMATETC@@0@Z
 0001:130A       ?SetData@CDataObject@@VEAPEXPEUtagFORMATETC@@PEUtagSTGMEDIUM@@H@Z
 0001:1328       ?EnumFormatEtc@CDataObject@@VEAPEXKPEPEUIEnumFORMATETC@@@Z
 0001:134E       ?EnumDAdvise@CDataObject@@VEAPEXPEPEUIEnumSTATDATA@@@Z
 0001:1390       ?QueryInterface@CExternalConnection@@VEAPEXAFUGUID@@PEPEX@Z
 0001:13CC       ?AddRef@CExternalConnection@@VEAKXZ
 0001:1400       ?Release@CExternalConnection@@VEAKXZ
 0001:1434       ?AddConnection@CExternalConnection@@VEAKKK@Z
 0001:146C       ?ReleaseConnection@CExternalConnection@@VEAKKKH@Z
 0001:14DA       ?QueryInterface@COleInPlaceActiveObject@@VEAPEXAFUGUID@@PEPEX@Z
 0001:1516       ?AddRef@COleInPlaceActiveObject@@VEAKXZ
 0001:154A       ?Release@COleInPlaceActiveObject@@VEAKXZ
 0001:157E       ?OnDocWindowActivate@COleInPlaceActiveObject@@VEAPEXH@Z
 0001:15AE       ?OnFrameWindowActivate@COleInPlaceActiveObject@@VEAPEXH@Z
 0001:15C8       ?GetWindow@COleInPlaceActiveObject@@VEAPEXPEI@Z
 0001:15F8       ?ContextSensitiveHelp@COleInPlaceActiveObject@@VEAPEXH@Z
 0001:1616       ?TranslateAccelerator@COleInPlaceActiveObject@@VEAPEXPEUtagMSG@@@Z
 0001:1632       ?ResizeBorder@COleInPlaceActiveObject@@VEAPEXPFUtagRECT@@PEUIOleInPlaceUIWindow@@H@Z
 0001:16B6       ?EnableModeless@COleInPlaceActiveObject@@VEAPEXH@Z
 0001:16D0       ?QueryInterface@COleInPlaceObject@@VEAPEXAFUGUID@@PEPEX@Z
 0001:1714       ?AddRef@COleInPlaceObject@@VEAKXZ
 0001:1748       ?Release@COleInPlaceObject@@VEAKXZ
 0001:177C       ?InPlaceDeactivate@COleInPlaceObject@@VEAPEXXZ
 0001:182A       ?UIDeactivate@COleInPlaceObject@@VEAPEXXZ
 0001:1854       ?SetObjectRects@COleInPlaceObject@@VEAPEXPFUtagRECT@@0@Z
 0001:19BC       ?GetWindow@COleInPlaceObject@@VEAPEXPEI@Z
 0001:19EC       ?ContextSensitiveHelp@COleInPlaceObject@@VEAPEXH@Z
 0001:1A0A       ?ReactivateAndUndo@COleInPlaceObject@@VEAPEXXZ
 0001:1A28       ?QueryInterface@COleObject@@VEAPEXAFUGUID@@PEPEX@Z
 0001:1A64       ?AddRef@COleObject@@VEAKXZ
 0001:1A98       ?Release@COleObject@@VEAKXZ
 0001:1ACC       ?SetClientSite@COleObject@@VEAPEXPEUIOleClientSite@@@Z
 0001:1B5A       ?Advise@COleObject@@VEAPEXPEUIAdviseSink@@PEK@Z
 0001:1BB6       ?SetHostNames@COleObject@@VEAPEXPFD0@Z
 0001:1BD0       ?DoVerb@COleObject@@VEAPEXJPEUtagMSG@@PEUIOleClientSite@@JIPFUtagRECT@@@Z
 0001:1D22       ?GetExtent@COleObject@@VEAPEXKPEUtagSIZEL@@@Z
 0001:1D9C       ?Update@COleObject@@VEAPEXXZ
 0001:1DC6       ?Close@COleObject@@VEAPEXK@Z
 0001:1DF4       ?Unadvise@COleObject@@VEAPEXK@Z
 0001:1E2E       ?EnumVerbs@COleObject@@VEAPEXPEPEUIEnumOLEVERB@@@Z
 0001:1E4A       ?GetClientSite@COleObject@@VEAPEXPEPEUIOleClientSite@@@Z
 0001:1E7E       ?SetMoniker@COleObject@@VEAPEXKPEUIMoniker@@@Z
 0001:1FB0       ?GetMoniker@COleObject@@VEAPEXKKPEPEUIMoniker@@@Z
 0001:2002       ?InitFromData@COleObject@@VEAPEXPEUIDataObject@@HK@Z
 0001:201E       ?GetClipboardData@COleObject@@VEAPEXKPEPEUIDataObject@@@Z
 0001:2048       ?IsUpToDate@COleObject@@VEAPEXXZ
 0001:2062       ?GetUserClassID@COleObject@@VEAPEXPEUGUID@@@Z
 0001:20A0       ?GetUserType@COleObject@@VEAPEXKPEPED@Z
 0001:20BC       ?SetExtent@COleObject@@VEAPEXKPEUtagSIZEL@@@Z
 0001:20DA       ?EnumAdvise@COleObject@@VEAPEXPEPEUIEnumSTATDATA@@@Z
 0001:211C       ?GetMiscStatus@COleObject@@VEAPEXKPEK@Z
 0001:2142       ?SetColorScheme@COleObject@@VEAPEXPEUtagLOGPALETTE@@@Z
 0001:215C       ?OpenEdit@COleObject@@RECXPEUIOleClientSite@@@Z
 0001:223C       ?QueryInterface@CPersistStorage@@VEAPEXAFUGUID@@PEPEX@Z
 0001:2278       ?AddRef@CPersistStorage@@VEAKXZ
 0001:22AC       ?Release@CPersistStorage@@VEAKXZ
 0001:22E0       ?InitNew@CPersistStorage@@VEAPEXPEUIStorage@@@Z
 0001:235A       ?GetClassID@CPersistStorage@@VEAPEXPEUGUID@@@Z
 0001:238A       ?Save@CPersistStorage@@VEAPEXPEUIStorage@@H@Z
 0001:23DA       ?SaveCompleted@CPersistStorage@@VEAPEXPEUIStorage@@@Z
 0001:24B0       ?Load@CPersistStorage@@VEAPEXPEUIStorage@@@Z
 0001:255E       ?IsDirty@CPersistStorage@@VEAPEXXZ
 0001:2578       ?HandsOffStorage@CPersistStorage@@VEAPEXXZ
 0001:259C       ?CreateStreams@CPersistStorage@@RECXPEUIStorage@@@Z
 0001:265A       ?OpenStreams@CPersistStorage@@RECXPEUIStorage@@@Z
 0001:2716       ?ReleaseStreamsAndStorage@CPersistStorage@@RECXXZ
 0001:27C0       ?CreateStreams@CPersistStorage@@RECXPEUIStorage@@PEPEUIStream@@1@Z
 0001:281C       ?QueryInterface@CSimpSvrObj@@VEAPEXAFUGUID@@PEPEX@Z
 0001:29A6       ?AddRef@CSimpSvrObj@@VEAKXZ
 0001:29E2       ?Release@CSimpSvrObj@@VEAKXZ
 0001:2A46       ??0CSimpSvrObj@@REC@PEVCSimpSvrDoc@@@Z
 0001:2CBA       ??1CSimpSvrObj@@REC@XZ
 0001:2D7E       ?Draw@CSimpSvrObj@@RECXIH@Z
 0001:2EFE       ?GetMetaFilePict@CSimpSvrObj@@RECIXZ
 0001:2FB8       ?SaveToStorage@CSimpSvrObj@@RECXPEUIStorage@@H@Z
 0001:315C       ?LoadFromStorage@CSimpSvrObj@@RECXXZ
 0001:321C       ?DoInPlaceActivate@CSimpSvrObj@@RECHJ@Z
 0001:34D2       ?AssembleMenus@CSimpSvrObj@@RECXXZ
 0001:358C       ?AddFrameLevelUI@CSimpSvrObj@@RECXXZ
 0001:3642       ?DoInPlaceHide@CSimpSvrObj@@RECXXZ
 0001:36F0       ?DisassembleMenus@CSimpSvrObj@@RECXXZ
 0001:374E       ?SendOnDataChange@CSimpSvrObj@@RECXXZ
 0001:37DE       ?DeactivateUI@CSimpSvrObj@@RECXXZ
 0001:389E       _TestDebugOut
 0001:38B6       WINMAIN
 0001:39FC       ?MainWndProc@@ZCJIIIJ@Z
 0001:3B3E       ?About@@ZCHIIGJ@Z
 0001:3B76       ?DocWndProc@@ZCJIIIJ@Z
 0001:3C22       __wflags
 0001:3C2C       __astart
 0001:3CE3       __nomain
 0001:3CEA       ??3@ZAXPEX@Z
 0001:3CFC       ??2@ZAPEXI@Z
 0001:3D0C       _abs
 0001:3D20       __fpurecall
 0001:3D20       __purecall
 0001:3D20       __npurecall
 0001:3D26       __dos_findnext
 0001:3D38       __dos_findfirst
 0001:3DB2       __aFlmul
 0001:3DB2       __aFulmul
 0001:3DE4       __fmemcmp
 0001:3E40       __fmemcpy
 0001:3E9E       __fmemset
 0001:3EE6       __aFftol
 0001:3EE6       __ftol
 0001:3F38       __stubmain
 0001:3F64       __cinit
 0001:4047       _exit
 0001:4055       __exit
 0001:4064       __cexit
 0001:4075       __c_exit
 0001:40E5       __ctermsub
 0001:4122       __FF_MSGBANNER
 0001:4146       __setargv
 0001:42F0       __setenvp
 0001:43AA       __cintDIV
 0001:43B4       __amsg_exit
 0001:43F6       __dosret0
 0001:4403       __dosreturn
 0001:4415       __dosretax
 0001:4427       __maperror
 0001:4454       __ffree
 0001:4475       __fmalloc
 0001:451C       __forcdecpt
 0001:4592       __cropzeros
 0001:4616       __positive
 0001:464E       __fassign
 0001:46A6       __cftoe
 0001:4872       __cftof
 0001:4A0A       __cftog
 0001:4AEA       __cfltcvt
 0001:4B8C       __fpsignal
 0001:4BB0       __wcexit
 0001:4BB0       __wcinit
 0001:4BB5       __wabout
 0001:4BB5       __wclose
 0001:4BB5       __wread
 0001:4BB5       __wopen
 0001:4BB5       __wsetsize
 0001:4BB5       __wterm
 0001:4BB5       __QWINMenuClick
 0001:4BB5       __QWINGetFocus
 0001:4BB5       __QWINTerm
 0001:4BB5       __QWINOpen
 0001:4BB5       __QWINInit
 0001:4BB5       __QWINGetBuffSize
 0001:4BB5       __QWINSetBuffSize
 0001:4BB5       __wgetsize
 0001:4BB5       __QWINRead
 0001:4BB5       __QWINClose
 0001:4BB5       __QWINIsQWINin
 0001:4BB5       __QWINGetSize
 0001:4BB5       __QWINSetAboutString
 0001:4BB5       __wsetfocus
 0001:4BB5       __QWINExit
 0001:4BB5       __wmenuclick
 0001:4BB5       __wgetfocus
 0001:4BB5       __QWINWrite
 0001:4BB5       __wsetscreenbuf
 0001:4BB5       __QWINSetSize
 0001:4BB5       __QWINSetFocus
 0001:4BB5       __QWINYield
 0001:4BB5       __wwrite
 0001:4BB5       __wgetscreenbuf
 0001:4BBC       __fptrap
 0001:4BC2       __NMSG_TEXT
 0001:4BF9       __NMSG_WRITE
 0001:4C36       __myalloc
 0001:4C64       __GetDGROUP
 0001:4C74       __searchseg
 0001:4CF0       __growseg
 0001:4D81       __incseg
 0001:4DE7       __findlast
 0001:4E08       __newseg
 0001:4E8A       _atof
 0001:4EE8       __fptostr
 0001:4F96       __fstrlen
 0001:4FB0       __fstrcpy
 0001:4FEC       __fmemmove
 0001:50B6       __fltout
 0001:510C       ___ExportedStub
 0001:5120       __initseg
 0001:5154       __linkseg
 0001:518A       _strlen
 0001:51A4       __aFahdiff
 0001:5212       $i8_output
 0001:5358       __fltin
 0001:5538       $i8_tpwr10
 0001:5576       __STRINGTOD
 0001:55DE       __STRINGTOLD
 0001:5AFE       __LD12MULTTENPOWER
 0001:5BD3       __LD12MULT
 0001:5D58       __MANTOLD12
 0001:5E20       ??_C@_0CB@GPOM@In?5CClassFactory?8s?5Constructor?$AN?6@
 0001:5E42       ??_7IClassFactory@@6F@
 0001:5E56       ??_7IUnknown@@6F@
 0001:5E62       ??_7CClassFactory@@6F@
 0001:5E76       ??_7CSimpSvrApp@@6F@
 0001:5E82       ??_7CSimpSvrDoc@@6F@
 0001:5E8E       ??_C@_0CA@JEOC@In?5CClassFactory?8s?5Destructor?$AN?6?$AA@
 0001:5EAE       ??0IOleWindow@@REC@XZ
 0001:5ED6       ??0IPersist@@REC@XZ
 0001:5EFE       ??_7IExternalConnection@@6F@
 0001:5F12       ??_7IPersistStorage@@6F@
 0001:5F3A       ??_7CDataObject@@6F@
 0001:5F6A       ??_7IDataObject@@6F@
 0001:5F9A       ??_7IOleInPlaceActiveObject@@6F@
 0001:5FC2       ??_7COleObject@@6F@
 0001:6022       ??_7CPersistStorage@@6F@
 0001:604A       ??_7IOleWindow@@6F@
 0001:605E       ??_7IOleObject@@6F@
 0001:60BE       ??_7COleInPlaceObject@@6F@
 0001:60E2       ??_7IPersist@@6F@
 0001:60F2       ??_7IOleInPlaceObject@@6F@
 0001:6116       ??_7CExternalConnection@@6F@
 0001:612A       ??_7CSimpSvrObj@@6F@
 0001:6136       ??_7COleInPlaceActiveObject@@6F@
 0001:615E       REGISTERHATCHWINDOWCLASS
 0001:61C4       CREATEHATCHWINDOW
 0001:620E       GETHATCHWIDTH
 0001:6232       GETHATCHRECT
 0001:62A6       SETHATCHRECT
 0001:630A       SETHATCHWINDOWSIZE
 0001:63D6       HATCHWNDPROC
 0001:64BA       ??_C@_0N@JEKA@Hatch?5Window?$AA@
 0001:64C8       ??_C@_0BG@FPGD@oleinplaceborderwidth?$AA@
 0001:64DE       ??_C@_07CIAP@windows?$AA@
 0001:64E6       OLEUIINITIALIZE
 0001:666A       OLEUIUNINITIALIZE
 0001:6682       PROMPTUSERDLGPROC
 0001:6728       UPDATELINKSDLGPROC
 0001:6AA6       ??_C@_0N@OCMF@VERIFICATION?$AA@
 0001:6AB4       ??_C@_0P@LMIA@OLEUI_MSG_HELP?$AA@
 0001:6AC4       ??_C@_0BE@FEHN@OLEUI_MSG_ENDDIALOG?$AA@
 0001:6AD8       ??_C@_0BB@PGGH@OLEUI_MSG_BROWSE?$AA@
 0001:6AEA       ??_C@_0BF@COIE@OLEUI_MSG_CHANGEICON?$AA@
 0001:6B00       ??_C@_0BD@HNAP@commdlg_FileNameOK?$AA@
 0001:6B14       ??_C@_0BK@LOCD@OLEUI_MSG_CLOSEBUSYDIALOG?$AA@
 0001:6B2E       ??_C@_0BC@GMEI@Object?5Descriptor?$AA@
 0001:6B40       ??_C@_0BH@FOOO@Link?5Source?5Descriptor?$AA@
 0001:6B58       ??_C@_0N@LHIH@Embed?5Source?$AA@
 0001:6B66       ??_C@_0BA@IEJA@Embedded?5Object?$AA@
 0001:6B76       ??_C@_0M@KPGD@Link?5Source?$AA@
 0001:6B82       ??_C@_09NJ@OwnerLink?$AA@
 0001:6B8C       ??_C@_08NJLM@FileName?$AA@
 0001:6B96       ??_C@_0M@MBIN@ole2uiRICls?$AA@
 0001:6BA2       ??_C@_0M@GHPL@ole2uiIBCls?$AA@
 0001:6BAE       ??_C@_0CG@HCKA@resource?5read?50x?$CFX?0?5my?5value?5is?5@
 0001:6BD4       ??_C@_00A@?$AA@
 0001:6BD6       ??_C@_03NAME@?4?4?4?$AA@
 0001:6BDA       ??_C@_09DKHB@Structure?$AA@
 0001:6BE4       ??_C@_04FOAE@?$CFd?$CF?$CF?$AA@
 0001:6BEA       XFORMWIDTHINPIXELSTOHIMETRIC
 0001:6C36       XFORMWIDTHINHIMETRICTOPIXELS
 0001:6C82       XFORMHEIGHTINPIXELSTOHIMETRIC
 0001:6CCE       XFORMHEIGHTINHIMETRICTOPIXELS
 0001:6D1A       XFORMRECTINPIXELSTOHIMETRIC
 0001:6DCA       PARSECMDLINE
 0001:6EE8       ??_C@_09LHIP@Embedding?$AA@
 0001:6EF2       _FIconBoxInitialize
 0001:6F68       _IconBoxUninitialize
 0001:6F6A       ICONBOXWNDPROC
 0001:70F4       OLEUIDRAWHANDLES
 0001:7322       OLEUIDRAWSHADING
 0001:74D8       OLESTDQUERYINTERFACE
 0001:7516       OLESTDGETDATA
 0001:7612       OLESTDMALLOC
 0001:7670       OLESTDFREE
 0001:76C6       OLESTDFREESTRING
 0001:771C       OLESTDCOPYSTRING
 0001:77A6       OLESTDCREATESTORAGEONHGLOBAL
 0001:783E       OLESTDCREATETEMPSTORAGE
 0001:789C       OLESTDGETOBJECTDESCRIPTORDATA
 0001:7A22       OLESTDVERIFYRELEASE
 0001:7A46       OLESTDRELEASE
 0001:7A6A       _OleStdNullMethod
 0001:7AEE       OLESTDGETFIRSTMONIKER
 0001:7BA4       OLESTDMARKPASTEENTRYLIST
 0001:7D4E       ??_C@_0DJ@NHNH@OleStdSwitchDisplayAspect?3?5Cache@
 0001:7D88       ??_C@_05FGFK@CLSID?$AA@
 0001:7D8E       ??_C@_09JJAI@Linked?5?$CFs?$AA@
 0001:7D98       ??_C@_07CPIP@Package?$AA@
 0001:7DA0       ??_C@_0CL@HONB@ERROR?3?5INTERFACE?5METHOD?5NOT?5IMPL@
 0001:7DCC       ??_C@_04MOFI@?$CFs?$CFd?$AA@
 0001:7DD2       ??_C@_0DC@GEMK@OleStdCreateTempFileMoniker?3?5Mon@
 0001:7E04       ??_C@_06KAHL@?$EA?$CFs?$CB?$CFs?$AA@
 0001:7E0C       _FResultImageInitialize
 0001:7EFC       _ResultImageUninitialize
 0001:7F0E       RESULTIMAGEWNDPROC
 0001:807E       _TransparentBlt
 0001:8208       OLEUIMETAFILEPICTICONFREE
 0001:8250       OLEUIMETAFILEPICTICONDRAW
 0001:8364       ENUMMETAFILEICONDRAW
 0001:83E0       ENUMMETAFILEEXTRACTLABEL
 0001:84BE       ENUMMETAFILEEXTRACTICON
 0001:86EA       ENUMMETAFILEEXTRACTICONSOURCE
 0001:87F0       OLESTDCOPYTARGETDEVICE
 0001:8842       OLESTDCOMPAREFORMATETC
 0001:8910       OLESTDCOMPARETARGETDEVICE
 0001:897A       ??_C@_07LGIJ@DISPLAY?$AA@
 0001:8AA4       OLESTDGETUSERTYPEOFCLASS
 0001:8C28       OLESTDGETDEFAULTFILEFORMATOFCLASS
 0001:8D06       ??_C@_08BJKM@CLSID?2?$CFs?$AA@
 0001:8D10       ??_C@_06HFAC@CLSID?2?$AA@
 0001:8D18       ??_C@_0BA@LJEI@?2AuxUserType?2?$CFd?$AA@
 0001:8D28       ??_C@_0M@BODG@?2MiscStatus?$AA@
 0001:8D34       ??_C@_0CB@FCAE@CLSID?2?$CFs?2DataFormats?2DefaultFile@
 0002:0004       rsrvptrs
 0002:0DD2       ?fBeVerbose@@3HE
 0002:0E10       _g_dwObjectCount
 0002:0E14       _g_dwLockCount
 0002:0E18       _uMsgHelp
 0002:0E1A       _uMsgEndDialog
 0002:0E1C       _uMsgBrowse
 0002:0E1E       _uMsgChangeIcon
 0002:0E20       _uMsgFileOKString
 0002:0E22       _uMsgCloseBusyDlg
 0002:0E50       _STKHQQ
 0002:0E52       __hPrevInstance
 0002:0E54       __hInstance
 0002:0E56       __lpszCmdLine
 0002:0E5A       __cmdShow
 0002:0E5C       _aseglo
 0002:0E5E       _aseghi
 0002:0E60       ___aDBswpflg
 0002:0E62       ___aDBrterr
 0002:0E64       __ctype_
 0002:0E64       __ctype
 0002:0F7A       __acfinfo
 0002:0F88       __aintdiv
 0002:0F8C       __fac
 0002:0F96       _errno
 0002:0F98       __umaskval
 0002:0F9A       __pspadr
 0002:0F9C       __psp
 0002:0F9E       __winver
 0002:0F9E       __winminor
 0002:0F9F       __winmajor
 0002:0FA0       __osminor
 0002:0FA0       __osver
 0002:0FA1       __osmajor
 0002:0FA2       __osversion
 0002:0FA4       __osmode
 0002:0FA5       __cpumode
 0002:0FA6       __oserr
 0002:0FA6       __doserrno
 0002:0FA8       __nfile
 0002:0FAA       __wfile
 0002:0FAC       __wnfile
 0002:0FAE       __osfile
 0002:0FC2       __wsfile
 0002:0FD6       ___argc
 0002:0FD8       ___argv
 0002:0FDC       __environ
 0002:0FE0       __pgmptr
 0002:0FE5       __child
 0002:0FE7       __exitflag
 0002:0FE8       __adbgmsg
 0002:1004       __pnhFarHeap
 0002:1008       __cfltcvt_tab
 0002:1024       __sigintseg
 0002:1026       __sigintoff
 0002:1028       __asizeC
 0002:1029       __asizeD
 0002:1036       __qwinused
 0002:1038       __fheap
 0002:1046       __amblksiz
 0002:10C4       __fpinit
 0002:14E2       ?lpCSimpSvrApp@@3PEVCSimpSvrApp@@E
 0002:14E2       _edata
 0002:14E2       __edata
 0002:14E6       ?lpClassFactory@@3PEUCClassFactory@@E
 0002:1F30       _cfEmbedSource
 0002:1F32       _cfEmbeddedObject
 0002:1F34       _ghInst
 0002:1F36       _cfOwnerLink
 0002:1F38       _cfLinkSrcDescriptor
 0002:1F3A       _cfFileName
 0002:1F3C       _cfLinkSource
 0002:1F3E       __mbac
 0002:1F46       _cfObjectDescriptor
 0002:1F48       __end
 0002:1F48       _end
 0000:4000  Abs  FJARQQ
 0000:5C32  Abs  FIDRQQ
 0000:8000  Abs  FJSRQQ
 0000:A23D  Abs  FIWRQQ
 0000:C000  Abs  FJCRQQ
 0000:FE32  Abs  FIARQQ

Program entry point at 0001:3c2c
